:020000040800F2
:1000000000280020050D0008490D0008490D0008D2
:10001000490D0008490D0008490D000800000000C6
:10002000000000000000000000000000490D000872
:10003000490D000800000000490D0008C90B000828
:10004000490D0008490D0008490D0008490D000838
:10005000490D0008490D0008490D0008490D000828
:10006000490D0008490D0008490D0008490D000818
:10007000490D0008490D0008490D0008490D000808
:10008000490D0008490D0008490D0008490D0008F8
:10009000490D0008490D0008490D0008490D0008E8
:1000A000490D0008490D0008490D0008490D0008D8
:1000B000490D0008490D000800000000490D000826
:1000C000490D00080000000000000000490D000874
:1000D00000000000490D0008490D00080000000064
:1000E000490D0008490D0008490D000800000000F6
:1000F0000000000000000000000000000000000000
:0C01000000000000000000005FF808F1A3
:10010C0080B483B000AF03463960FB7197F90730B8
:10011C00002B0BDA0D49FB7903F00F03043B3A6813
:10012C00D2B21201D2B20B441A7609E0084997F9FF
:10013C0007303A68D2B21201D2B20B4483F80023D2
:10014C0000BF0C37BD4680BC704700BF00ED00E01F
:10015C0000E100E080B582B000AF78607B68B3F15D
:10016C00807F01D3012311E00A4A7B6823F07F438F
:10017C00013B53600F214FF0FF30FFF7C1FF054BE0
:10018C0000229A60034B07221A6000231846083796
:10019C00BD4680BD10E000E080B500AF154A154BA0
:1001AC001B6843F0010313601249124B5A68124B3F
:1001BC0013404B600F4A0F4B1B6823F0847323F4DE
:1001CC00803313600B4A0B4B1B6823F480231360A2
:1001DC00084A084B5B6823F4FE035360054B4FF44D
:1001EC001F029A6000F078F8044B4FF000629A609E
:1001FC0000BF80BD001002400000FFF800ED00E0E1
:10020C0080B485B000AF0023FB600023BB600023EB
:10021C007B602C4B5B6803F00C03FB60FB68042BCE
:10022C0007D0082B09D0002B33D1274B274A1A6053
:10023C0033E0254B254A1A602FE0224B5B6803F410
:10024C007013BB601F4B5B6803F480337B60BB682F
:10025C009B0C0233BB607B68002B06D1BB681C4A2D
:10026C0002FB03F3184A136017E0164B5B6803F4A8
:10027C000033002B06D0BB68154A02FB03F3124A6D
:10028C0013600AE0BB68114A02FB03F30E4A1360C9
:10029C0003E00D4B0D4A1A6000BF0A4B5B6803F07C
:1002AC00F0031B090B4AD35CDBB2FB60064B1A68EC
:1002BC00FB6822FA03F3044A136000BF1437BD46EF
:1002CC0080BC7047001002400000002000127A0031
:1002DC0000093D000400002080B500AF00F002F8DA
:1002EC0000BF80BD80B483B000AF00237B600023CF
:1002FC003B603A4A394B1B6843F480331360374BED
:10030C001B6803F400333B607B6801337B603B6804
:10031C00002B03D17B68B3F5A06FF0D12F4B1B687A
:10032C0003F40033002B02D001233B6001E00023D7
:10033C003B603B68012B4BD1294A294B1B6843F08E
:10034C0010031360264A264B1B6823F0030313602B
:10035C00234A234B1B6843F0020313601F4A1F4BB5
:10036C005B6853601D4A1D4B5B6853601B4A1B4BFB
:10037C005B6843F480635360184A184B5B6823F442
:10038C007C135360154A154B5B6843F4E8135360B8
:10039C00124A124B1B6843F08073136000BF0F4B63
:1003AC001B6803F00073002BF9D00C4A0B4B5B68F5
:1003BC0023F003035360094A084B5B6843F00203C4
:1003CC00536000BF054B5B6803F00C03082BF9D19D
:1003DC0000BF0C37BD4680BC704700BF0010024008
:1003EC000020024080B485B000AF78600B467B8063
:1003FC000023FB737B681B899AB27B8813409BB2EA
:10040C00002B02D00123FB7301E00023FB73FB7B69
:10041C0018461437BD4680BC704700BF80B483B00B
:10042C0000AF78600B467B807B687A889A8100BF2E
:10043C000C37BD4680BC704780B483B000AF786089
:10044C007B689B899BB218460C37BD4680BC7047B5
:10045C0080B582B000AF0346FB7100BF02210E488D
:10046C00FFF7C0FF0346002BF8D0FB799BB219466F
:10047C000948FFF7D3FF00BF01210748FFF7B2FF80
:10048C000346002BF8D00448FFF7D6FF0346DBB237
:10049C0018460837BD4680BD0030014080B489B095
:1004AC0000AF786039600023FB6100233B610023BF
:1004BC00BB610023FB6000237B610023BB603B68B6
:1004CC00DB7803F00F03FB613B68DB7803F0100370
:1004DC00002B05D03B689B781A46FB691343FB61E4
:1004EC003B681B88DBB2002B44D07B681B687B61AC
:1004FC000023BB6138E00122BB6902FA03F3FB6005
:10050C003B681B881A46FB6813403B613A69FB68E1
:10051C009A4226D1BB699B00FB600F22FB6802FA52
:10052C0003F3BB60BB68DB437A6913407B61FA69F8
:10053C00FB6802FA03F37A6913437B613B68DB784F
:10054C00282B05D10122BB699A407B685A6108E0CF
:10055C003B68DB78482B04D10122BB699A407B684D
:10056C001A61BB690133BB61BB69072BC3D97B68BB
:10057C007A691A603B681B88FF2B46D97B685B68DD
:10058C007B610023BB613AE0BB690833012202FAAC
:10059C0003F3FB603B681B881A46FB6813403B6106
:1005AC003A69FB689A4227D1BB699B00FB600F221A
:1005BC00FB6802FA03F3BB60BB68DB437A69134048
:1005CC007B61FA69FB6802FA03F37A6913437B6176
:1005DC003B68DB78282B05D1BB69083301229A4094
:1005EC007B685A613B68DB78482B05D1BB690833C3
:1005FC0001229A407B681A61BB690133BB61BB69FC
:10060C00072BC1D97B687A695A6000BF2437BD4675
:10061C0080BC704780B485B000AF7860396000232F
:10062C00FB817B681B88FB81FB8903F44153FB81B5
:10063C003B681A883B685B8813439AB23B689B887B
:10064C0013439AB23B68DB8813439AB23B681B890D
:10065C0013439AB23B685B8913439AB23B689B89FC
:10066C0013439AB23B68DB8913439AB2FB89134359
:10067C00FB817B68FA891A807B689B8B9BB223F485
:10068C0000639AB27B689A833B681A8A7B681A82E9
:10069C0000BF1437BD4680BC704700BF80B483B028
:1006AC0000AF78600B46FB70FB78002B08D07B68A2
:1006BC001B889BB243F040039AB27B681A8007E018
:1006CC007B681B889BB223F040039AB27B681A802C
:1006DC0000BF0C37BD4680BC704700BF80B483B0F0
:1006EC0000AF78600B467B807A887B681A6100BF0C
:1006FC000C37BD4680BC704780B483B000AF7860C7
:10070C000B46FB70FB78002B06D00949084B9A6905
:10071C007B6813438B6106E00549054B9A697B683E
:10072C00DB4313408B6100BF0C37BD4680BC704768
:10073C000010024080B483B000AF78600B467B8021
:10074C007A887B685A6100BF0C37BD4680BC704705
:10075C0080B586B000AF01210420FFF7CDFF012149
:10076C004FF48050FFF7C8FFE023BB820323BB7517
:10077C001823FB7507F1140319461748FFF78EFE73
:10078C001023BB821023FB7507F114031946124882
:10079C00FFF784FE00233B804FF482737B800023A1
:1007AC00BB800223FB8001233B814FF400737B81D0
:1007BC000823BB810023FB8107233B823B46194660
:1007CC000648FFF727FF01210448FFF767FF00BF2A
:1007DC001837BD4680BD00BF000801400030014005
:1007EC0080B500AF10211848FFF7A4FF9522002117
:1007FC00002000F02BF8012000F05EF80346002BDF
:10080C0001D0FF231DE010210F48FFF767FFFF20E9
:10081C00FFF71EFE10210C48FFF78CFFFF22002172
:10082C00012000F013F8002000F046F80346002BDE
:10083C00E9D110210448FFF751FFFF20FFF708FE14
:10084C000023184680BD00BF0008014080B586B06B
:10085C0000AF03463960FB711346BB7100237B610B
:10086C00FB7943F04003DBB23B733B681B0EDBB2FE
:10087C007B733B681B0CDBB2BB733B681B0ADBB2A4
:10088C00FB733B68DBB23B74BB797B7400237B61ED
:10089C000AE007F10C027B6913441B781846FFF73A
:1008AC00D7FD7B6901337B617B69052BF1D900BFD7
:1008BC001837BD4680BD00BF80B584B000AF03467D
:1008CC00FB7140F6FF73FB6002E0FB68013BFB60D1
:1008DC0000F012F803461A46FB79934202D0FB68EB
:1008EC00002BF2D1FB68002B01D1FF2300E0002389
:1008FC0018461037BD4680BD80B582B000AF0023CE
:10090C00FB7100BF02210E48FFF76CFD0346002B64
:10091C00F8D0FF210A48FFF781FD00BF01210848EC
:10092C00FFF760FD0346002BF8D00548FFF784FD68
:10093C000346FB71FB7918460837BD4680BD00BFE6
:10094C000030014080B582B000AF00237B601EE018
:10095C00FFF7D2FF0346FB70FB7803F01F03FB701D
:10096C00FB780B2B06D00D2B06D0052B06D10523BF
:10097C00BB7006E00B2316E00D2314E0FF23BB70C5
:10098C0000BFBB78052B06D07B6801337B607B688E
:10099C00402BDDD900E000BF00BFFFF7ADFF0346E1
:1009AC00002BFAD0FB7818460837BD4680BD00BF37
:1009BC0080B582B000AF00237B60FFF7C9FE102129
:1009CC000A48FFF78BFE00237B6005E0FF20FFF752
:1009DC003FFD7B6801337B607B68092BF6D9FFF701
:1009EC00FFFE034618460837BD4680BD000801408F
:1009FC0080B500AF094B1B88002B01D100230AE006
:100A0C00FFF7D6FF03469AB2044B1A80034B1B88A0
:100A1C00002BF5D10123184680BD00BF1800002023
:100A2C0080B500AF00BFFFF7E3FF0346002BFAD100
:100A3C0000BF80BD80B584B000AF78603B4B1A78A6
:100A4C003B4B1A70394B00221A700023FB60FF23BA
:100A5C00FB7210213748FFF76DFEFF2279681820D2
:100A6C00FFF7F4FE0020FFF727FF0346002B4ED1C3
:100A7C00FF20FFF7EDFCFE20FFF7EAFC2C4B1B7868
:100A8C00012B1AD10023FB6014E02B4AFB6832F8CF
:100A9C001330DBB21846FFF7DBFC274AFB6832F851
:100AAC0013301B0A9BB2DBB21846FFF7D1FCFB6874
:100ABC000133FB60FB68FF2BE7D91D4B1B78022B26
:100ACC001AD10023FB6014E01C4AFB6832F8133087
:100ADC00DBB21846FFF7BCFC184AFB6832F813303F
:100AEC001B0A9BB2DBB21846FFF7B2FCFB68013362
:100AFC00FB60FB68FF2BE7D9FFF7FEFEFFF7FCFE60
:100B0C00FFF720FF0346052B01D10023FB721021B8
:100B1C000848FFF7E3FDFF20FFF79AFC044B002287
:100B2C001A70FB7A18461037BD4680BD300600207F
:100B3C001B0000200008014030020020300400207F
:100B4C0080B500AFFFF734FF03461A46144B1A600A
:100B5C00FFF766FF134B00221A80134B4FF4007201
:100B6C001A60FFF74DFB114B1B68114AA2FB0323C4
:100B7C005B0B1846FFF7EEFA0E4B1B78002BFBD0E5
:100B8C000D4B01221A70084B1B681846FFF752FFD9
:100B9C00054B1B6803F50073034A1360ECE700BFB9
:100BAC001400002026020020280200200000002053
:100BBC005917B7D1300600203206002080B400AFA0
:100BCC00404B1B78012B29D13F4B1B78012B25D097
:100BDC003E4BB1221A803E4B1B781A463D4B19886E
:100BEC003D4B23F812103A4B1B780133DAB2384BD9
:100BFC001A70374B1B781A46344B1B8899B2364BFC
:100C0C0023F81210324B1B780133DAB2304B1A70C6
:100C1C00304B1B8801339AB22E4B1A80294B1B7810
:100C2C00022B29D1284B1B78022B25D0274BB22223
:100C3C001A80274B1B781A46264B1988274B23F80A
:100C4C001210234B1B780133DAB2214B1A70204B54
:100C5C001B781A461D4B1B8899B2204B23F8121097
:100C6C001B4B1B780133DAB2194B1A70194B1B88CA
:100C7C0001339AB2174B1A80154B1B78FE2B0CD1F3
:100C8C00104B1B78012B08D10E4B02221A70144BFF
:100C9C0001221A700E4B00221A700D4B1B78FE2B82
:100CAC000CD1084B1B78022B08D1064B01221A7071
:100CBC000B4B02221A70064B00221A7000BFBD4665
:100CCC0080BC70471A0000201B0000202C02002062
:100CDC0031060020340600203002002030040020B1
:100CEC00300600204C0D0008000000201C000020E5
:100CFC001C00002038060020002103E00A4B5B5842
:100D0C004350043109480A4B42189A42F6D3094A17
:100D1C0002E0002342F8043B074B9A42F9D3FFF759
:100D2C003BFAFFF70DFF70474C0D00080000002048
:100D3C001C0000201C00002038060020FEE70000EC
:100D4C0000A24A040000000000000000010203049D
:0C0D5C00060708090A000000FFFF010262
:0400000508000D05DD
:00000001FF
